:040000000200BE320A
:01000B0032C2
:0100130032BA
:01001B0032B2
:0100230032AA
:03002B000200339D
:0B00BE007581201200BAE58260030289
:0200C900002E07
:0800CB007900E94400601B7A92
:0500D300009001067819
:0C00D8000075A000E493F2A308B8000239
:0900E40005A0D9F4DAF275A0FFC1
:0800ED007800E84400600C7982
:0D00F50000900000E4F0A3D8FCD9FAF6D882
:01010200FDFF
:0301030002002EC9
:05002E0012008B80FEB2
:0E003300C0E0C0F0C082C083C0D075D018D32A
:0400410010AF01C338
:07004500C0D010CF02803093
:0A004C000520907F98E0FA30E214DE
:07005600C3E5209414401FD4
:0D005D00907F98E0FA54FBF07520008012AF
:07006A00C3E5209450400B98
:0B007100907F98E0FA4404F075200036
:0E007C00D0D092AFD0D0D083D082D0F0D0E0E0
:01008A003243
:0D008B00C2AF75200075C80075CDB175CBF2
:0E009800B175CCE075CAE0D2ADC2CFD2CA902D
:0E00A6007F9EE0FA4404F0907F98E0FA54FB4D
:0300B400F0D2AFD8
:0200B70080FEC9
:0100B9002224
:0300BA007582004C
:0100BD002220
:00000001FF
